S0220000687474703A2F2F737265636F72642E736F75726365666F7267652E6E65742F1D
S12300000C9438000C94EB1A0C942F210C945F000C945F000C945F000C945F000C945F0074
S12300200C945F000C943D240C945F000C94DA270C945F000C943D1B0C94C51A0C94971956
S12300400C94DA280C945F000C9459280C945F000C9479290C9441290C945F000C945F0091
S12300600C945F000C945F000C945F000C945F0011241FBECFEFD0E1DEBFCDBF14BEA895C7
S123008088E10FB6F89480936000109260000FBE13E0A0E0B1E0ECE6F6E502C005900D92B9
S12300A0A83EB107D9F718E0A8EEB3E001C01D92A335B107E1F70E944F130C94352B0C9431
S12300C0000020E030E0D901A859BD4F0E94172B802DF901E85DF94F80832F5F3F4F81E08D
S12300E02034380781F720E030E0D901A857BE4F0E94172B802DF901E45CFE4F80832F5F52
S12301003F4F2530310589F712BC11BC089520E030E0F901E85DF94F8081D901A859BD4F8B
S1230120082E0E94242B2F5F3F4F81E02034380781F712BC11BC089520E030E0D901509604
S12301400E94172B802DF901E854FB4F80832F5F3F4F81E02034380789F712BC11BC0895BF
S123016020E030E0F901E854FB4F8081D9015096082E0E94242B2F5F3F4F81E020343807F3
S123018089F712BC11BC089520E430E0D901A05BBE4F0E94172B802DF901ED5BFE4F80838A
S12301A02F5F3F4F203A310589F712BC11BC089520E430E0F901ED5BFE4F8081D901A05B5E
S12301C0BE4F082E0E94242B2F5F3F4F203A310589F712BC11BC0895A2E0B0E00E94172B8D
S12301E0802D90E090931E0180931D0120911D0130911E01A3E0B0E00E94172B802D90E0A8
S1230200982F8827820F931F90931E0180931D01ADEEB3E00E94172B802D90E09093220139
S1230220809321012091210130912201AEEEB3E00E94172B802D90E0982F8827820F931FE5
S1230240909322018093210180911D0190911E019093200180931F01A4E0B0E00E94172B41
S1230260802D90E090932401809323012091230130912401A5E0B0E00E94172B802D90E00D
S1230280982F8827820F931F9093240180932301A6E0B0E00E94172B802D90E090930101E6
S12302A0809300012091000130910101A7E0B0E00E94172B802D90E0982F8827820F931FE0
S12302C09093010180930001A1E0B0E00E94172B802D8093E803A8E0B0E00E94172B802D98
S12302E080931301A9E5B1E00E94172B802D80932D01A2E0B4E00E94172B902D892F8150A2
S1230300843078F080912D01843039F481E08093180183E68093FC0506C082E0809318013F
S123032002C090931801A9E0B0E00E94172B802D80931201AEE0B0E00E94172B802D809329
S12303402601ABE0B0E00E94172B802D80931901A3E0B4E00E94172B802D80931A01ACE037
S1230360B0E00E94172B802D80931B01AFE6B1E00E94172B802D80931C01A2EFB1E00E947E
S1230380172B802D80935D0480915D04882319F081E080935D04ADE0B0E00E94172B802D4D
S12303A026E0829FC00111249093150180931401A1E7B1E00E94172B802D80932006A0E751
S12303C0B1E00E94172B802D80931E068AE080938D0781E080938B07AFE8B1E00E94172B9D
S12303E0802D80932E0180912E0181FF05C080912E01827F80932E0180912E0185FF05C079
S123040080912E018F7280932E01A4EFB1E00E94172B802D90E02CE231E0AC01429FC001C2
S1230420439F900D529F900D11249093B7048093B604A5EFB1E00E94172B802D8093B3044B
S1230440A6EFB1E00E94172B802D8093B104A7EFB1E00E94172B802D8093B004A8EFB1E072
S12304600E94172B802D90E09093AF048093AE042091AE043091AF04A9EFB1E00E94172BF8
S1230480802D90E0982F8827820F931F9093AF048093AE04ABEFB1E00E94172B802D90E0BB
S12304A09093300180932F0120912F0130913001ACEFB1E00E94172B802D90E0982F88272B
S12304C0820F931F9093300180932F01ADEFB1E00E94172B802D90E0909332018093310175
S12304E02091310130913201AEEFB1E00E94172B802D90E0982F8827820F931F90933201E3
S123050080933101AFEFB1E00E94172B802D90E090937603809375032091750330917603D8
S1230520A0E0B2E00E94172B802D90E0982F8827820F931F909376038093750320E030E0B4
S1230540D901A25ABE4F0E94172B802DF901ED51FE4F8083D901AE58BE4F0E94172B802D1D
S1230560F901E350FA4F8083D901A458BE4F0E94172B802D808B2F5F3F4F2A30310501F7DB
S1230580A7E0B2E00E94172B802D80933701A3E0B2E00E94172B802D8093380120E030E060
S12305A0F901E659F84F84E6808BD901A45EBD4F0E94172B802D80832F5F3F4F2031310523
S12305C079F720E030E0D901A759BE4F0E94172B802DF901E85DFE4F80832F5F3F4F243020
S12305E0310589F720E030E0D901A25DBD4F0E94172B802DF901E654FC4F80832F5F3F4F1D
S12306002031310589F7ADE6B1E00E94172B802D80932501A1EFB1E00E94172B802D80931C
S12306205C04A0EFB1E00E94172B802D80932C01A6E0B2E00E94172B802D8093270120E081
S123064030E0D901AA54BC4F0E94172B802DF901E351FE4F80832F5F3F4F2031310589F771
S1230660A7ECB3E00E94172B802D80933A01A8ECB3E00E94172B802D80933B01A4EDB3E046
S12306800E94172B802D80936804A5EDB3E00E94172B802D80936904A6EDB3E00E94172B06
S12306A0802D80936A04A7EDB3E00E94172B802D80936B04A8EDB3E00E94172B802D809302
S12306C06C04A9EDB3E00E94172B802D80936D04AAEDB3E00E94172B802D80936E04ABED90
S12306E0B3E00E94172B802D80936F04A8EEB3E00E94172B802D90E0909334018093330183
S12307002091330130913401A9EEB3E00E94172B802D90E0982F8827820F931F90933401BE
S123072080933301AAEEB3E00E94172B802D80935F04ACECB3E00E94172B802D2AE0829F55
S1230740C00111249093770480937604A1EDB3E00E94172B802D829FC001112490937C0408
S123076080937B04A2EDB3E00E94172B802D829FC001112490937E0480937D0412BC11BC45
S1230780089580911D0190911E01A2E0B0E0082E0E94242B80911D0190911E01892F992729
S12307A0A3E0B0E0082E0E94242B8091230190912401A4E0B0E0082E0E94242B8091230110
S12307C090912401892F9927A5E0B0E0082E0E94242B8091000190910101A6E0B0E0082E9A
S12307E00E94242B8091000190910101892F9927A7E0B0E0082E0E94242B80911301A8E06C
S1230800B0E0082E0E94242B80911201A9E0B0E0082E0E94242B12BC11BC089580E0A1EF91
S1230820B1E0082E0E94242B8AE0A0EFB1E0082E0E94242B80915D04A2EFB1E0082E0E94DF
S1230840242B84E0A9E5B1E0082E0E94242B85E0ACE0B0E0082E0E94242B82E3AFE6B1E068
S1230860082E0E94242B24E1A1E7B1E0022E0E94242B91E0A0E7B1E0092E0E94242B88ECE9
S1230880A4EFB1E0082E0E94242BA5EFB1E0092E0E94242BA6EFB1E0022E0E94242B8AE506
S12308A0A7EFB1E0082E0E94242B88EEA8EFB1E0082E0E94242B83E0A9EFB1E0082E0E94BD
S12308C0242B80912F0190913001ABEFB1E0082E0E94242B80912F0190913001892F9927D5
S12308E0ACEFB1E0082E0E94242B8091310190913201ADEFB1E0082E0E94242B8091310173
S123090090913201892F9927AEEFB1E0082E0E94242B8091750390917603AFEFB1E0082E2A
S12309200E94242B8091750390917603892F9927A0E0B2E0082E0E94242B8CEDA7E0B2E05C
S1230940082E0E94242B86EEA3E0B2E0082E0E94242B2CE132E088ECD901082E0E94242B28
S12309602F5F3F4F82E02C323807A9F782E2AFE8B1E0082E0E94242B81E0A6E0B2E0082E56
S12309800E94242B12BC11BC0895CF92DF92EF92FF920F931F93CF93DF93C0E0D0E0A5E049
S12309A0B2E00E94172B202D30E040E050E0A3EDB3E00E94172B602D6E01CC0CDD1C8DEFC0
S12309C091E0C80ED91EF601E080F18070E080E090E00E94882A00E010E0A80197010E94E6
S12309E0882A24E630E040E050E00E94DA2A79018A01CA01B90124EF31E040E050E00E9491
S1230A00882A28EC30E040E050E0E20EF31E041F151FA80197010E94DA2ACA01B9012FEFCA
S1230A2030E040E050E00E94882A25E030E040E050E00E94DA2AE2E0220F331F441F551FD7
S1230A40EA95D1F7CA01B90124E630E040E050E00E94DA2AF601318320832196C732D105E2
S1230A6009F09DCFC0E0D0E0A9ECB3E00E94172B202D30E040E050E0A3EDB3E00E94172BFD
S1230A80602D6E01CC0CDD1C8BE492E0C80ED91EF601E080F18070E080E090E00E94882A9B
S1230AA000E010E0A80197010E94882A24E630E040E050E00E94DA2A79018A01CA01B90133
S1230AC024EF31E040E050E00E94882A28EC30E040E050E0E20EF31E041F151FA80197013D
S1230AE00E94DA2ACA01B9012FEF30E040E050E00E94882A25E030E040E050E00E94DA2AEA
S1230B0092E0220F331F441F551F9A95D1F7CA01B90124E630E040E050E00E94DA2AF60182
S1230B20318320832196C732D10509F09DCFC0E0D0E0AAECB3E00E94172B202D30E040E095
S1230B4050E0A3EDB3E00E94172B602D6E01CC0CDD1C89E992E0C80ED91EF601E080F18014
S1230B6070E080E090E00E94882A00E010E0A80197010E94882A24E630E040E050E00E948C
S1230B80DA2A79018A01CA01B90124EF31E040E050E00E94882A28EC30E040E050E0E20E97
S1230BA0F31E041F151FA80197010E94DA2ACA01B9012FEF30E040E050E00E94882A25E086
S1230BC030E040E050E00E94DA2A02E0220F331F441F551F0A95D1F7CA01B90124E630E0C9
S1230BE040E050E00E94DA2AF601318320832196C732D10509F09DCFC0E0D0E0A4E0B2E05C
S1230C000E94172B202D30E040E050E0A3EDB3E00E94172B602D6E01CC0CDD1C87EE92E084
S1230C20C80ED91EF601E080F18070E080E090E00E94882A00E010E0A80197010E94882A42
S1230C4024E630E040E050E00E94DA2A79018A01CA01B90124EF31E040E050E00E94882A2E
S1230C6028EC30E040E050E0E20EF31E041F151FA80197010E94DA2ACA01B9012FEF30E00A
S1230C8040E050E00E94882A25E030E040E050E00E94DA2AB2E0220F331F441F551FBA9566
S1230CA0D1F7CA01B90124E630E040E050E00E94DA2AF601318320832196C732D10509F006
S1230CC09DCFDF91CF911F910F91FF90EF90DF90CF900895EAE7F0E0108280E280937C00E7
S1230CE080E880BF87EE808311B885E090E09093F7038093F60388E790E09093EB03809307
S1230D00EA0384E690E09093F9038093F803909301048093000486E490E09093FB0380938E
S1230D20FA0308950F931F93CF93DF93282F30E0F901EE0FFF1FEE5FFE4F0081118143E0A1
S1230D40033F140718F0E2E3F0E04CC053E00F3D150718F0EAE0F0E045C0C0E0D0E087E28E
S1230D6090E0A901489F9001499F300D589F300D1124D901AC0FBD1FAA0FBB1FA350BE4F4B
S1230D808D919C9111978017910730F5FE013197E20FF31FEE0FFF1FE350FE4F2081318150
S1230DA0608171814D915C91FE01EE0FFF1FEE0FFF1FEC0FFD1F3596201B310BC901880FA2
S1230DC0991F880F991F641B750B820F931F0E94B32AE60FF71F06C02196C732D10549F6B1
S1230DE0E8ECF0E0CF01DF91CF911F910F9108950F931F93CF93DF93AC01E0E0F0E0EF0169
S1230E00CC0FDD1FDE01AB5CBC4F8D919C91119748175907C0F56D917C913197EE0FFF1FB1
S1230E20DF01AB5CBC4F8D919C911197681B790B8D919C91C35BDC4F28813981E35BFC4F42
S1230E4000811181481B590B84E690E0DC014A9FC0014B9F900D5A9F900D11240E94B32A82
S1230E60201B310B0190F081E02D629FC001639F900D729F900D112464E670E00E94B32A8B
S1230E806E0F7F1F09C03196EA30F10509F0B7CF6091610370916203CB01DF91CF911F910D
S1230EA00F9108958091EA039091EB03282F205527FF0AC08091140190911501BC01660F99
S1230EC0771F680F791F1EC02F312CF0609114017091150117C040911401509115013327E4
S1230EE027FD309588E290E0821B930B9C01249FC001259F900D349F900D11246AE070E02F
S1230F000E94B32ACB0108950F931F93CF93DF93AC0180917803909179034817590718F41C
S1230F20E0EFF0E057C080919403909195038417950718F4E0E0F0E04DC0E1E0F0E0EF0135
S1230F40CC0FDD1FDE01A858BC4F8D919C91119748175907C0F56D917C913197EE0FFF1F77
S1230F60DF01A858BC4F8D919C911197681B790B8D919C91EA56FC4F20813181CA56DC4F14
S1230F8008811981481B590B84E690E0DC014A9FC0014B9F900D5A9F900D11240E94B32A31
S1230FA0201B310B0190F081E02D629FC001639F900D729F900D112464E670E00E94B32A4A
S1230FC0E61BF70B07C03196EE30F10509F0B7CFEEEFF0E0CF01DF91CF911F910F910895AF
S1230FE080917404882359F08CED95E0909336018093350110928904109288042AC0809187
S12310007404882349F08CED95E0909336018093350184E690E019C080917404882349F0BF
S12310208CED95E090933601809335018AEF90E00CC080917404882361F08CED95E09093D0
S123104036018093350184EF91E09093890480938804F89480915804909159048A5A9A4A9A
S1231060C1F080915804909159048555954589F0789480916807909169078064909369070F
S12310808093680784EF91E090933601809335010AC0789480916807909169078F7B90932F
S12310A0690780936807F89480915A0490915B048F3F89F078948091680790916907806873
S12310C0909369078093680784EF91E090933601809335010AC07894809168079091690789
S12310E08F7790936907809368078091350190913601892B99F12F9A2091880430918904A0
S12311002115310511F42F9A16C08091860490918704029780F485B1881F8827881F80951F
S123112087958827879595B19F77982B95B9309387042093860480918604909187040197ED
S1231140909387048093860480913501909136010197909336018093350108952F98109260
S1231160890410928804089580916807909169079F779093690780936807809100019091A4
S1231180010197FD44C08091E80380FF32C020914F043091500480911F01909120018C59D3
S12311A09F4F8217930720F461E070E040E832C020914F043091500480911F0190912001BF
S12311C049978217930720F461E070E048E022C020914F043091500480911F0190912001BD
S12311E0845690408217930790F461E070E044E011C020914F043091500480911F01909199
S123120020018217930718F460E070E802C060E070E040E02091680730916907CB01992783
S1231220869597958827822B932B90936907809368072091680730916907CB01807090781F
S1231240822B932B9093690780936807809100019091010192FF33C020914F043091500438
S123126080912F01909130018217930740F520914F04309150048091310190913201281780
S12312803907E8F42091F6033091F7038091250190E001962817390794F4809168079091E3
S12312A06907946090936907809368078091E80380FF03C0616048600BC0706809C080918D
S12312C06807909169079B7F90936907809368072091F8033091F9038091380190E082171F
S12312E0930734F480913801882311F060614860809169042091FA033091FB0390E08F5B84
S12313009F4F8217930774F480916904882351F0606280914F0490915004895B9B40A0F0EC
S1231320446012C0809169042091FA033091FB0390E0C296821793073CF4809169048823F4
S123134019F0606251E001C050E080916804209100043091010490E0C296821793076CF449
S123136080916804882349F0606480914F0490915004855C994008F0446080916A042091E5
S1231380FE033091FF0390E0C2968217930734F480916A04882311F06068446080916B044B
S12313A02091FC033091FD0390E0C2968217930734F480916B04882311F0606844608091EC
S12313C06C04209102043091030490E0880F991F8217930734F480916C04882311F060680B
S12313E0446080916D04209104043091050490E0880F991F8217930734F480916D048823F9
S123140011F06068446080916E04209106043091070490E0880F991F8217930734F4809126
S12314206E04882311F06068446080916F04209108043091090490E0880F991F821793071D
S123144034F480916F04882311F060684460552321F082E380934B0402C010924B04189B0E
S123146006C060FD02C077FF09C06170707870937204609371044093730406C01092720482
S12314801092710410927304409374040895809100019091010193FF1FC11A9B06C08091FD
S12314A07A048F5F80937A0402C010927A0480917A04853108F454C01092750420914F04D5
S12314C03091500480917503909176038217930778F4809171049091720482609093720499
S12314E0809371048091730488608093730409C080917104909172048D7F909372048093C8
S123150071048091E80383FF16C080914F0490915004815D974078F08091710490917204EB
S1231520846090937204809371048091730482608093730409C080917104909172048B7FBE
S123154090937204809371048091760490917704909379048093780484E380937A04B1C0A7
S12315608091780490917904892B09F45DC08091780490917904019790937904809378047C
S123158080917504823099F0833030F4882351F0813009F096C019C08330A9F1843009F0EC
S12315A090C031C010927904109278048AC08091710490917204846090937204809371043D
S12315C08091730482608093730420914F043091500480917503909176038217930768F448
S12315E080917104909172048260909372048093710480917304886059C080917104909197
S123160072048D7F0CC090918F0480917703891708F440C080917104909172048B7F909353
S12316207204809371044DC04E9B20C080914F04909150048D5D9540C8F0809184049091C8
S123164085040196909385048093840420917B0430917C0428173907A0F580917D049091E7
S12316607E04909383048093820414C0209182043091830421153105E1F080914F0490918C
S123168050048D5D9540A8F021503040309383042093820480917104909172048460909313
S12316A07204809371048091730482608093730408C010928504109284041092830410924C
S12316C082048091730481FF07C080912E0180FF03C084E68093B20408959C018091E803C6
S12316E084FF1BC022533040C901F3E0880F991FFA95E1F7220F331F280F391F2455354F41
S1231700442737FD4095542F60E579E784E090E00E94FC2A822F90E008958091E80385FD51
S123172003C084E690E0089522533040C90173E0880F991F7A95E1F7220F331F280F391F21
S12317402455354F442737FD4095542F60E579E784E090E00E94FC2A2C592695822F90E0EF
S12317600895A89582E50E94CE2983E10E94CE2980914F0490915004892F99270E94CE29A4
S123178080914F04909150040E94CE2980910004909101040E94CE2980918F040E94CE29C2
S12317A08091EA039091EB030E94CE298091F8039091F9030E94CE298091F6039091F70398
S12317C00E94CE298091F2039091F3030E94CE2980915604909157046091180170E00E94D3
S12317E0B32ACB010E94CE29809153049091540420915504F4E096958795FA95E1F7807F37
S1231800822B0E94CE2980915304909154040E94CE2920916807309169078091F805909184
S1231820F905E3E096958795EA95E1F78170232F3327822B0E94CE29809168079091690751
S12318400E94CE298091AF0780950E94CE2980918A070E94CE298091F0039091F1030E9480
S1231860CE298091FA059091FB05969587950E94CE298091B2079091B3079093030480937A
S123188002048091920790919307909305048093040420918C0430E0220F331FF901E6508E
S12318A0FC4F80819181892F990F990BB3E0220F331FBA95E1F7822B0E94CE29E0918C043E
S12318C0F0E0EE0FFF1FE650FC4F808191810E94CE298DEA0E94CE2980918C048F5F80933A
S12318E08C04883010F010928C040895CF92DF92EF92FF920F931F93CF93DF93A89588E11B
S12319000FB6F89480936000109260000FBE0E941A2A882309F4B9C60E94AB2990938B04FB
S123192080938A048336910509F4BBC38436910508F049C08035910509F482C4813591050D
S123194008F58134910509F4CCC08234910568F48932910509F4D5C58433910509F47CC696
S12319608832910509F08FC6A9C58634910509F4DAC18D34910509F48EC28534910509F083
S123198082C626C18735910509F4D1C48835910568F48335910509F406C68535910509F41D
S12319A013C58235910509F06EC6C6C48136910509F44DC08236910508F070C38835910524
S12319C009F061C649C58037910509F43EC481379105E8F48736910509F40AC488369105ED
S12319E048F48536910509F4C9C28636910508F056C15AC38D36910509F40CC28F369105D1
S1231A0009F442C58936910509F03DC6CAC3853F910509F466C1863F910568F48937910555
S1231A2009F492C58A37910509F496C38837910509F029C691C3873F910571F1873F9105F6
S1231A4008F4ACC1883F910509F01DC685C081E60E94CE2980EA0E94CE2910928B041092C5
S1231A608A040EC0E85DF94F80810E94CE2980918A0490918B04019690938B0480938A04A6
S1231A80E0918A04F0918B04E03AF10558F382E30E941F298EE9F7C587EF0E94CE2980EADD
S1231AA00E94CE2910928B0410928A040EC0E853F94F80810E94CE2980918A0490918B04EE
S1231AC0019690938B0480938A04E0918A04F0918B04E03AF10558F382E30E941F2988E0F7
S1231AE0D2C510928B0410928A0400E010E00E941A2A882349F1C0918A04D0918B04C03A86
S1231B00D10591F40E94AB2990938B0480938A048E3B910519F406E11AEF16C0E091800476
S1231B20F0918104099510C00E94AB29C85DD94F888380918A0490918B04019690938B04C7
S1231B4080938A0400E010E00F5F1F4F4AEF0030140708F09AC5CBCF10928B0410928A045E
S1231B60C0E0D0E00E941A2A882359F100918A0410918B04003A110589F40E94AB29909381
S1231B808B0480938A04079719F4C6E1DAEF19C0E0918004F0918104099513C000561F4FED
S1231BA00E94AB29085D194FF801808380918A0490918B04019690938B0480938A04C0E009
S1231BC0D0E02196FAEFC030DF0708F05EC5CACFC0E0D0E00E941A2A882309F459C00E948E
S1231BE0AB298A3B910509F050C588E10FB6F89480936000109260000FBE10928B041092D5
S1231C008A043EC0885B0E94CE298DEF0E94CE2920918A0430918B048AEF90E0289FE00183
S1231C20299FD00D389FD00D112407C0DE010E94172B802D0E94CE29219620918A0430918B
S1231C408B042F5F3F4F8AEF90E0AC01249FC001259F900D349F900D112421503040C817F5
S1231C60D90720F3822F885B80950E94CE2980918A0490918B04019690938B0480938A04F2
S1231C8080918A0490918B048430910508F4BACF21965AEFC030D50708F0F7C49BCF86E6CD
S1231CA00E94CE2980EA0E94CE2910928B0410928A040EC0E854FB4F80810E94CE29809124
S1231CC08A0490918B04019690938B0480938A04E0918A04F0918B04E03AF10558F389E9FC
S1231CE0D2C485EF0E94CE2980EA0E94CE2910928B0410928A040EC0E85AFA4F80810E94DD
S1231D00CE2980918A0490918B04019690938B0480938A04E0918A04F0918B04E03AF10570
S1231D2058F38AE0B0C410928B0410928A0400E010E00E941A2A882349F1C0918A04D0913A
S1231D408B04C03AD10591F40E94AB2990938B0480938A04893B910519F406E11AEF16C0A5
S1231D60E0918004F0918104099510C00E94AB29C854DB4F888380918A0490918B04019649
S1231D8090938B0480938A0400E010E00F5F1F4F8AEF0030180708F078C4CBCF10928B0479
S1231DA010928A04C0E0D0E00E941A2A882359F100918A0410918B04003A110589F40E9406
S1231DC0AB2990938B0480938A04099719F4C6E1DAEF19C0E0918004F0918104099513C076
S1231DE000561F4F0E94AB2908541B4FF801808380918A0490918B04019690938B04809338
S1231E008A04C0E0D0E02196FAEFC030DF0708F03CC4CACF8DE60E94CE2989E00E94CE29CB
S1231E2080911D0190911E010E94CE2980911D0190911E01892F99270E94CE2980912301E1
S1231E40909124010E94CE298091230190912401892F99270E94CE298091000190910101DE
S1231E600E94CE298091000190910101892F99270E94CE29809113010E94CE29809112019D
S1231E800E94CE29AAE0B0E00E94172B802D0E94CE2982E9F8C310928B0410928A04C0E03A
S1231EA0D0E00E941A2A8A3008F461C00E94AB2990931E0180931D0100911D0110911E0159
S1231EC00E94AB29982F8827800F911F90931E0180931D010E94AB2990932401809323016B
S1231EE000912301109124010E94AB29982F8827800F911F90932401809323010E94AB2943
S1231F00909301018093000100910001109101010E94AB29982F8827800F911F90930101FF
S1231F20809300010E94AB29809313010E94AB29809312010E94AB29AAE0B0E0082E0E94E8
S1231F40242B0E94F2230E94AB29823B910551F40E94C103E0918004F09181040995CFE6B5
S1231F60DAEF05C0E0918004F0918104099521964AEFC030D40708F088C393CF85E60E94C9
S1231F80CE2983E10E94CE2910928B0410928A040EC0ED51FE4F80810E94CE2980918A0456
S1231FA090918B04019690938B0480938A04E0918A04F0918B04EA30F10558F380911901EE
S1231FC00E94CE2980911B010E94CE2983E00E942029809128010E94CE29809129010E94A0
S1231FE0CE2980912A010E94CE2980912B010E94CE29809114019091150166E070E00E94A6
S1232000B32ACB010E94CE29809125010E94CE29AEE6B1E00E94172B802D0E94CE298AE9E8
S12320200E94CE298CE60E94CE2984E10E94CE2910928B0410928A040EC0E350FA4F80814E
S12320400E94CE2980918A0490918B04019690938B0480938A04E0918A04F0918B04EA3081
S1232060F10558F310928B0410928A040EC0E350FA4F80890E94CE2980918A0490918B047F
S1232080019690938B0480938A04E0918A04F0918B04EA30F10558F383E9F5C20E9487009C
S12320A0F4C20E94B000F1C281E50E94CE2980E10E94CE298091B6039091B7030E94CE292A
S12320C08091990790919A070E94CE2980919B0790919C070E94CE2980919D0790919E0765
S12320E00E94CE2980919F079091A0070E94CE298091A1079091A2070E94CE298091A30754
S12321009091A4070E94CE298091F2039091F3030E94CE29809173040E94CE2980917104F9
S1232120909172040E94CE298091AF0780950E94CE2980918F040E94CE2980911D060E94E3
S1232140CE2984E00E94CE2985E00E94CE2986E00E94CE298EEA97C20E94B10B96C20E9461
S1232160AB29C82FD0E00E94AB29C817D90709F08CC20E94AB298C0190938B0480938A040E
S12321800E94AB290817190709F07FC20E94AB298639910509F079C280918A04C85DD94F61
S12321A04DC00E941A2A8530D0F6FBCF0E94AB29C82FD0E00E94AB29C817D90709F065C271
S12321C00E94AB298C0190938B0480938A040E94AB290817190709F058C20E94AB298839A6
S12321E0910509F052C280918A04C854DB4F26C00E941A2A8530D0F6FBCF0E94AB29C82FD5
S1232200D0E00E94AB29C817D90709F03EC20E94AB298C0190938B0480938A040E94AB2910
S12322200817190709F031C20E94AB298F3A910509F02BC280918A04CD5BDE4F888325C2CE
S12322400E941A2A8530C8F6FBCFC0E0D0E00E941A2A823080F10E94AB290E94AB298F384B
S1232260910509F012C210928B0410928A041CC0ED5BFE4F108180E70E94CE2982E00E9490
S1232280CE2980918A040E94CE29812F0E94CE298FE80E94CE2980918A0490918B040196CC
S12322A090938B0480938A04E0918A04F0918B04E03AF105E8F221965AEFC030D50709F405
S12322C0E4C1C5CF0E94AB298C010E94AB29D82FCC27C00FD11F0E94AB298C0190938B04DA
S12322E080938A040E94AB290817190709F0CDC10E94AB29883A9105A9F4DE010E941F2BC7
S1232300E07080918A0490918B04E82BF92BF0938B04E0938A04DE010F010E94302B12BC16
S123232011BCB3C1E0918004F091810409950E941A2A853038F6FBCFCC24DD240E941A2A55
S12323408330C0F10E94AB298C010E94AB29EC010E94AB298D3A910509F097C1FC2EEE244F
S1232360E00EF11ED7010E94172B802D90E0D70111960E94172B002D10E0102F0027080F86
S1232380191F84E50E94CE2984E00E94CE29802F0E94CE298E2D0E94CE29EF2CFF248E2D6D
S12323A00E94CE29012F1127802F0E94CE298BEA0E94CE290894C11CD11C80E0C8168AEFA5
S12323C0D80609F462C1BACFCC24DD240E941A2A8330C0F10E94AB298C010E94AB29EC01D1
S12323E00E94AB298A3A910509F04FC1FC2EEE24E00EF11ED7010E94172B802D90E0D70116
S123240011960E94172B002D10E0102F0027080F191F85E50E94CE2984E00E94CE29802FAC
S12324200E94CE29012F1127802F0E94CE298E2D0E94CE29EF2CFF248E2D0E94CE298AEAF5
S12324400E94CE290894C11CD11CE0E0CE16EAEFDE0609F41AC1BACFC0E0D0E00E941A2A81
S1232460882359F00E94AB29873A910509F00DC1E0918004F091810409952196FAEFC030A7
S1232480DF0709F402C1EACFC0E0D0E00E941A2A882369F00E94AB298039910509F0F5C02C
S12324A00E94D800E0918004F0918104099521964AEFC030D40709F4E8C0E8CFC0E0D0E09E
S12324C00E941A2A8823B1F00E94AB29873D910509F0DBC08091F6039091F703ADE6B1E019
S12324E0082E0E94242B12BC11BCE0918004F0918104099521965AEFC030D50709F4C5C02F
S1232500DFCFC0E0D0E00E941A2A8823B1F00E94AB29863D910509F0B8C08091F60390911C
S1232520F703AEE6B1E0082E0E94242B12BC11BCE0918004F0918104099521968AEFC030FD
S1232540D80709F4A2C0DFCFC0E0D0E00E941A2A823010F10E94AB29892B09F096C00E9487
S1232560AB2986389105C1F489E70E94CE2985E00E94CE298FEC0E94CE298FE30E94CE2954
S123258081E10E94CE298DE20E94CE298EE00E94CE2986E80E94CE292196EAEFC030DE07C1
S12325A009F473C0D3CFC0E0D0E00E941A2A823008F44CC00E94AB29892B09F047C00E9489
S12325C0AB298C3A910509F060C083E50E94CE2988E00E94CE2980915804909159040E941F
S12325E0CE298091580490915904892F99270E94CE2980912606909127060E94CE298091AF
S1232600260690912706892F99270E94CE2980912106909122060E94CE29809121069091B8
S12326202206892F99270E94CE298091B5079091B6070E94CE298091B5079091B607892FB6
S123264099270E94CE298CEA0E94CE292196FAEFC030DF07D1F0A9CFC0E0D0E00E941A2A29
S1232660823058F00E94AB29892B79F40E94AB298B3C910511F40E94EC0021964AEFC0307F
S1232680D40719F0EBCF0E94CE29A895DF91CF911F910F91FF90EF90DF90CF9008950F9387
S12326A01F93CF93DF9310926907109268070E9417293D9A3E9A3C9A459A469A449A3F9A90
S12326C0479A38984098399841983A9842983B984398389839983A983B9854985C98559856
S12326E05D9854985598239A269A279A2B9A2E982F98259A249A53985298229856982198C5
S123270020980E942229AAE5B1E00E94172B802D80935E040E949D230E94F2230E94052901
S12327200E946A060E94C5042B9A2E98A7E0B0E00E94172B802D12BC11BC85FF9BC080915A
S12327400001909101019F7D90930101809300010E94C1030E940E040E94B0000E94870067
S12327600E94D80086E0AAE0B0E0082E0E94242B89E1ABE0B0E0082E0E94242B8EE1ACE08D
S1232780B0E0082E0E94242BAEE0B0E0082E0E94242B20E030E0F901ED51FE4F8081D901C9
S12327A0A25ABE4F082E0E94242B2F5F3F4F2A30310589F780912801A9E6B1E0082E0E9487
S12327C0242B80912901AAE6B1E0082E0E94242B80912A01ABE6B1E0082E0E94242B80918D
S12327E02B01ACE6B1E0082E0E94242B20E030E0F901E350FA4F8081D901AE58BE4F082EB5
S12328000E94242B2F5F3F4F2A30310589F720E030E0F901E350FA4F8089D901A458BE4F25
S1232820082E0E94242B2F5F3F4F2A30310589F780912006A1E7B1E0082E0E94242B8091B9
S123284014019091150166E070E00E94B32AADE0B0E0062E0E94242B84E1ADE6B1E0082E12
S12328600E94242B81EEAEE6B1E0082E0E94242B12BC11BC0E94C4000E94EC000E949C00DB
S12328800E946100809100019091010185FD07C080916F008B7F80936F00459A469A8091D7
S12328A02701882311F480E801C080E4809339011092E90380911401909115018D5A9D40B3
S12328C030F08CEA9DE0909315018093140110924C0486B3866086BB78948AEA0E94CE2915
S12328E080E00E94CE2985E50E94CE2983B1869581708093600480916E00836080936E003E
S12329002B9A2E9AA89580914F04909150048635910570F180914C04882351F5809168078C
S1232920909169079F7E909369078093680780916F00856080936F0080916E008360809374
S12329406E002B9A81E080934C0480916807909169078062909369078093680780916807F4
S1232960909169079062909369078093680749C080914C04813009F044C080914F0490911E
S123298050048234910508F03CC080916F008D7F80936F00809170008C7F80937000809171
S12329A06F008B7F80936F0080916E00836080936E0080916807909169078F7D9093690785
S12329C0809368078091680790916907877F9093690780936807389839983A983B98549813
S12329E05598459A469A449A10924C0480916807909169079F7D9093690780936807109273
S1232A004A0480914C048130D9F480916F00826080936F00809170008360809370008091A9
S1232A206E00836080936E008091680790916907886090936907809368072B9A2E9A14C051
S1232A4010924A04459A469A449A10924A041092B300109257041092560480914101909133
S1232A604201892B09F42B988091E903833009F4DCC0843018F4882371F077C0853009F49D
S1232A80DBC1853008F442C1863009F4C1C1873009F086C210C280914D0490914E04853653
S1232AA0910508F480C2E091E903F0E080917800909179008C7F65E070E00E94B32AEE0FD2
S1232AC0FF1FE65DFB4F718360838091E903C82FD0E0E091E903F0E0EE0FFF1FE651FC4F02
S1232AE080819181E091E903F0E0EE0FFF1FE65DFB4F20813181880F991F880F991F820F68
S1232B00931F880F991F6AE070E00E94B32ACC0FDD1FC651DC4F7983688310924E04109201
S1232B204D048091E9038F5F8093E9038091E903806480937C000E94760C0E9452079093A4
S1232B401701809316018091410190914201892B09F45CC180914101909142010197909338
S1232B604201809341012B9A51C180914D0490914E048536910508F416C29091E90340910A
S1232B807004842F83708450990F990F980FE92FF0E0EE0FFF1FEE5FFE4F808191812091EB
S1232BA0780030917900820F931F969587959183808310924E0410924D04A8958091E9039D
S1232BC0C42FD0E08130D1F48E01085F1F4F842F0E949206000F111F06511C4FF801918379
S1232BE08083809170048823A9F48091FA039091FB030E946D0B80938E070CC08081918133
S1232C0062E070E00E94C72ACC0FDD1FCE5FDB4F798368838091E9038F5F8093E90380917B
S1232C20E903806480937C00BEC180914D0490914E048536910508F4B6C1E091E903F0E0EC
S1232C4080917800909179009695879596958795EE0FFF1FE65DFB4F918380838091E90303
S1232C60C82FD0E0E091E903F0E0EE0FFF1FE651FC4F80819181E091E903F0E0EE0FFF1F84
S1232C80E65DFB4F20813181880F991F880F991F820F931F880F991F6AE070E00E94B32A07
S1232CA0CC0FDD1FC651DC4F7983688310924E0410924D048091E9038F5F8093E90380912E
S1232CC0E90390913901892B80937C000E94760CA895809170048F5F80937004843010F057
S1232CE01092700420917004922F91709295990F907E85B18F7D892B85B9220F220F220F2F
S1232D00207185B18F7E822B85B94DC180914D0490914E048159914008F445C18091270127
S1232D20882329F1E091E903F0E080917800909179009695879596958795EE0FFF1FE65D8E
S1232D40FB4F91838083A091E903B0E0E091E903F0E0EE0FFF1FE65DFB4F80819181AA0FC0
S1232D60BB1FA651BC4F11969C938E933EC0E091E903F0E08091780090917900EE0FFF1F13
S1232D80E65DFB4F918380838091E903C82FD0E0E091E903F0E0EE0FFF1FE651FC4F00819C
S1232DA01181E091E903F0E0EE0FFF1FE65DFB4F808191810E9484079C01220F331F280F11
S1232DC0391FC80143E0880F991F4A95E1F7801B910B820F931F6AE070E00E94B32ACC0F37
S1232DE0DD1FC651DC4F7983688310924E0410924D048091E9038F5F8093E9038091E903DC
S1232E00806880937C008091600483B1A895CBC080914D0490914E048536910508F4C3C021
S1232E20E091E903F0E0809178009091790096958795969587950FC080914D0490914E040C
S1232E40893C910508F4AFC0E091E903F0E08091780090917900EE0FFF1FE65DFB4F91839C
S1232E608083A091E903B0E0E091E903F0E0EE0FFF1FE651FC4F20813181E091E903F0E054
S1232E80EE0FFF1FE65DFB4F80819181820F931F96958795AA0FBB1FA651BC4F11969C937E
S1232EA08E9310924E0410924D048091E9038F5F8093E9036DC080914D0490914E0485365F
S1232EC0910508F470C0E091E903F0E08091780090917900969587959695879590E0EE0FE1
S1232EE0FF1FE65DFB4F91838083E091E903F0E0EE0FFF1FE651FC4F8081918184369105DF
S1232F000CF5A091E903B0E0E091E903F0E0EE0FFF1FE651FC4F40815181E091E903F0E075
S1232F20EE0FFF1FE65DFB4F20813181CA01880F991F840F951F820F931F9695879596957C
S1232F40879519C0A091E903B0E0E091E903F0E0EE0FFF1FE651FC4F20813181E091E90351
S1232F60F0E0EE0FFF1FE65DFB4F80819181820F931F96958795AA0FBB1FA651BC4F1196FC
S1232F809C938E9310924E0410924D041092E9038091E903806480937C000E94760C36CFCF
S1232FA081E08093E90380914D0490914E04019690934E0480934D0480914F04909150048F
S1232FC08752924008F452C08091BB0787FF02C0E0E002C0E091BB0780918C078F5F8093BF
S1232FE08C0790918C0780918D07981708F441C010928C072091F8033091F9034E2F50E0EA
S1233000FA01E659F84F808190E02817390754F480918A07843634F480918A0790918B071A
S1233020890F13C02091F8033091F903FA01E659F84F808190E0281739074CF080918A0769
S123304082302CF080918A07815080938A0720918A07FA01E659F84F8089332727FD309578
S123306090E0821793072CF4808901C081E080938A0780914F04909150048739910508F48F
S12330806DC02091F6033091F7038091250190E04996281739070CF061C08091B40490918E
S12330A0B50401969093B5048093B4042091B4043091B5048091B6049091B704281739070C
S12330C008F440C01092B5041092B40420914F04309150048091AE049091AF040A972817AB
S12330E0390730F49091B2048091B304890F15C020914F04309150048091AE049091AF04AC
S123310049968217930758F49091B2048091B104891728F48091B20481508093B204909172
S1233120B2048091B004891718F48091B00408C09091B2048091B104981720F48091B104B1
S12331408093B20480914F04909150048A58924038F48091B0048093B20402C01092B20441
S12331608091E80382FF4FC080914F0490915004855F914008F447C080914F049091500455
S1233180805D974008F03FC02091F6033091F7038091250190E0059628173907A4F5209110
S12331A0F6033091F7038091630490E00196821793074CF18091640490916504A0916604CA
S12331C0B09167040196A11DB11D8093640490936504A0936604B093670480916404909130
S12331E06504A0916604B09167048158994AA340B04010F181E08093620480916807909110
S12332006907916015C08091F6039091F70380936304109264041092650410926604109212
S123322067041092620480916807909169079E7F90936907809368070E94B4080E94470A83
S12332400E94F007809100019091010180FF67C080912E0180FF11C08091AD04883C28F0C8
S12332608091B2048823B9F418C09091B2048091AD048695891790F010C080912E0182FFEE
S12332800DC08091AD04883C48F0809168079091690796FF02C0549A01C0549880912E015C
S12332A084FF16C08091AD04883C28F080918A0718165CF12CC020918A078091AD043327AC
S12332C027FD3095869590E0821793070CF11FC080912E0186FF1CC08091AD04883CC0F090
S12332E020914F043091500480913301909134018217930760F42091F8033091F903809115
S12333005F0490E08217930714F4559A01C055988091AD04883C28F01092AD0402C054985F
S123332055988091AD048F5F8093AD04EACA1F920F920FB60F9211248F939F938091BC075F
S12333408F5F8093BC078091BC07882309F447C0809168079091690790619093690780937A
S1233360680710924C0480916807909169079F7D909369078093680780916F008B7F809309
S12333806F0080916F008D7F80936F00809170008C7F8093700080916E00836080936E00BA
S12333A0459A469A449A80916807909169078F7D9093690780936807809168079091690729
S12333C0877F9093690780936807389839983A983B98549855981092500410924F047894B8
S12333E09F918F910F900FBE0F901F9018952091B9073091BA0780918400909185002817A5
S12334003907F0F4809195078630A1F480915A0490915B04880F991F90935B0480935A045B
S123342080915A0490915B04816090935B0480935A0404C010925B0410925A0481E003C0DC
S1233440809195078F5F8093950780918400909185009093BA078093B9070895282F809127
S123346068079091690793FD0BC0223031F0233031F0213029F445980895469808954498C7
S123348008951F938091A504882309F45CC08091A5048130A1F4459A1092A5048091B40369
S12334A09091B5039093C5078093C40780914F04909150048559914198F182E02FC08091EE
S12334C0A5048230A1F4469A1092A5048091B4039091B5039093AE078093AD0780914F0429
S12334E09091500485599141D8F083E017C08091A5048330A9F4449A1092A5048091B403A6
S12335009091B5039093BE078093BD0780914F04909150048559914118F081E00E942E1A33
S12335208091210690912206892B69F18091B707882349F1809121069091220690938B0015
S123354080938A0020C08091B7078823E1F01091B707113041F01091B707123021F010917B
S1233560B707133031F48091B7070E942E1A1093A5048091B5079091B60790938B008093B0
S12335808A001092B7071F9108951F920F920FB60F9211242F933F934F935F936F937F9387
S12335A08F939F93AF93BF93EF93FF930E94411A2B9A7894FF91EF91BF91AF919F918F914D
S12335C07F916F915F914F913F912F910F900FBE0F901F9018951F920F920FB60F92112423
S12335E02F933F934F935F936F937F938F939F93AF93BF93EF93FF938091B4039091B503AE
S123360001969093B5038093B4038091E80387FF23C08091A6048823F9F02091B40330918D
S1233620B503809192079091930748E750E0BA01681B790B2617370769F02091B40330914B
S1233640B5038091B2079091B307481B590B2417350711F40E94411AFF91EF91BF91AF9129
S12336609F918F917F916F915F914F913F912F910F900FBE0F901F9018951F920F920FB608
S12336800F9211248F939F93F89480919607882309F486C0809171049091720497FD80C0E3
S12336A08091130180958093AF078091AF0790911D068C59891B8093AF079091FC059430C0
S12336C029F1953040F4923051F19330B8F4913009F058C009C09731C1F1933609F441C084
S12336E09E3009F04FC023C08091AF078093B20084E08093B100389A83E050C08091AF074D
S123370086BD83E085BD3A9A84E048C08091AF078093B2009093B1003B9A82E03FC08091D6
S1233720AF0786BD83E085BD399A81E037C081E08093D1038091AF078093B20084E0809371
S1233740B100389A3B9A87E129C081E08093D2038091AF0786BD83E085BD399A3A9A8EE0AF
S12337601DC081E08093D1038091AF078093B20084E08093B100389A3B9A3A9A399A9093FB
S1233780FC050EC08091AF078093B20084E08093B100389A3B9A3A9A399A83E68093FC05D7
S12337A078949F918F910F900FBE0F901F901895CF93DF93EC0180915D04E7E0F0E0E81B75
S12337C0F109EE0FFF1FE651FC4F8081918120915C04821B482F50E080912C0126E0829F81
S12337E0C00111249C01249FC001259F900D349F900D112464E670E00E94B32A603A71057F
S123380020F08FE98093B80702C06093B8078091B8076AE00E94A72A8093910780919107F5
S123382080311CF08FE08093910780914F0490915004885E934008F0AAC010928F078FEF03
S12338408093BB078091910724E18202C0011124909354048093530480914F0490915004A9
S123386064E670E00E94B32A65506093B40780914F0490915004845F914060F41092B4078A
S1233880E091B407FF27E7FDF095E45CFE4F808190E0A9C08091B4078430E1F5E0915304E4
S12338A0F0915404E85DF94F2081E091B407FF27E7FDF095E45CFE4F6081E091B407FF2782
S12338C0E7FDF095E45CFE4F808190E09093FB058093FA05E091FA05F091FB0580914F04F3
S12338E0909150044091B40730E0220F331F261B3109845F91406CE94602A0011124840FFB
S1233900951FAC01249FC001259F900D349F900D11243AC0E091B407FF27E7FDF095E35CC4
S1233920FE4F6081E091B407FF27E7FDF095E45CFE4F4081E091B407FF27E7FDF095E45C51
S1233940FE4F808190E09093FB058093FA05E091FA05F091FB0580914F04909150042091F5
S1233960B40770E0641B7109845F91404CE9240290011124820F931F9C01629FC001639FC6
S1233980900D729F900D112464E670E0D3C080914F0490915004875F924250F187EC80931C
S12339A08F0780918F076AE00E94A72A8093BB07809191072091BB0744E18402C001112477
S12339C0332727FD3095820F931F9093540480935304E0915304F0915404E85DF94F808149
S12339E090E0880F991F9093FB058093FA05AAC080914F0490915004885E934062E370E03E
S1233A000E94B32A60938F0780918F076AE00E94A72A8093BB07809191072091BB0744E120
S1233A208402C0011124332727FD3095820F931F9093540480935304E0915304F0915404FA
S1233A40E85DF94F808190E0880F991F9093FB058093FA058091BB0787FD38C08091BB07BE
S1233A608331A4F5E0915304F0915404E75DF94F6081E0915304F0915404E85DF94F5081E8
S1233A80E091FA05F091FB0580918F072091BB0790E04AE0240290011124821B930B880FBF
S1233AA0991F70E0651B7109AC01469FC001479F900D569F900D11246AE070E00E94C72A36
S1233AC0E60FF71FF093FB05E093FA058091910787FD38C0809191078F30A4F5E0915304F4
S1233AE0F0915404E45CF94F6081E0915304F0915404E85DF94F5081E091FA05F091FB0590
S1233B008091B8072091910790E04AE0240290011124821B930B880F991F70E0651B71092E
S1233B209C01269FC001279F900D369F900D11246AE070E00E94C72AE60FF71FF093FB0599
S1233B40E093FA058091680790916907977F90936907809368078091F8059091F905877F80
S1233B609093F9058093F80580917304882309F458C08091730488233CF180917304883028
S1233B8088F08091940790E083709070892B09F448C08091940767E00E94A72A992309F4C2
S1233BA040C012C0809173048430C0F08091940790E083709070892B39F08091940767E064
S1233BC00E94A72A992369F580916807909169079860909369078093680723C080917304CB
S1233BE0823050F08091F8059091F90588609093F9058093F80515C080917304882389F008
S1233C008091FA059091FB058739910550F08091FA059091FB058C5890409093FB058093BE
S1233C20FA05809194078F5F8093940740918F04445645310CF044E18091FA059091FB0573
S1233C4020911201885B9F4F820F911D6AE070E00E94B32A7093B3076093B20780914F04A6
S1233C60909150042091B2073091B30768E270E00E94B32A260F311D3093930720939207A1
S1233C802091FA053091FB058091120190914B04285B3F4F280F311D291B3109842F4C3ECA
S1233CA00CF48CEE992787FD9095280F391F30938E0420938D0480918D0490918E048D5BB8
S1233CC092402CF06CEB72E080E090E015C080918D0490918E0405972CF465E070E080E09E
S1233CE090E00AC080918D0490918E04AC01BA01882777FD8095982F2091510430915204AD
S1233D002C0F3D1F40E050E00E94882A20EB34E040E050E00E94DA2AC21BD30BCE01DF9155
S1233D20CF910895A0E0B0E0BC01CD0128E532E040E050E00E94882A20EB34E040E050E0B5
S1233D400E94DA2ADA01C90108950F931F93CF93DF938091CA039091CB039093C307809382
S1233D60C2078091CA039091CB03499708F471C28091BC07882349F088EE9DEF9093CF03EB
S1233D808093CE031092BC0753C080914F04909150044091CE035091CF03895B9B40C0F026
S1233DA0E0915104F09152042091CA033091CB038091B80390E0241B350BAC01429FC0014B
S1233DC0439F900D529F900D112464E170E017C0E0915104F09152042091CA033091CB0387
S1233DE08091B80390E0241B350BAC01429FC001439F900D529F900D11246EE170E00E9432
S1233E00C72ACB018E0F9F1F62E070E00E94C72A70935204609351041092520410925104D1
S1233E208091CA039091CB039093CF038093CE0380914A04893628F480914A048F5F80933E
S1233E404A0480914F0490915004C091CE03D091CF03D0932706C093260620912606309135
S1233E6027060091CC031091CD0340E050E060E070E489E191E00E94FC2ACA01B90124E12F
S1233E8030E040E050E00E94882A20EC30E0A901049F9001059F300D149F300D11242050FA
S1233EA0324040E050E00E94DA2A3093500420934F0480914F04909150048D5D954010F0E1
S1233EC0E8981AC0E89A80914F04909150048C54944090F48091B6039091B70387379105F8
S1233EE058F08091B6039091B7038A37910520F481E08093A60402C01092A60420919C04E9
S1233F0030919D0440919A0450919B04C901880F991F820F931F840F951F96958795969537
S1233F20879590939D0480939C04809198049091990490939B0480939A0480919604909140
S1233F409704909399048093980480919404909195049093970480939604809192049091BD
S1233F60930490939504809394048091900490919104909393048093920480914F049091FC
S1233F805004909391048093900480914F04909150048D5D9540B8F080918F044091900421
S1233FA05091910420919C0430919D0490E0821B930B840F951F9695879596958795855B74
S1233FC080938F040FC084E680938F04809151049091520464E070E00E94C72A70935204FB
S1233FE0609351041092BC0780914F04909150048C529140A0F58091CC039091CD03039788
S123400071F580919507813051F584E090E09093CD038093CC038091CC039091CD03806830
S123402080938100809184009091850096958795969587959093850080938400D695C79519
S1234040D695C795D093CF03C093CE03809126069091270696958795969587953AC0809118
S12340604F0490915004875B9340B8F18091CC039091CD03049789F580919507813069F570
S123408083E090E09093CD038093CC038091CC039091CD0380688093810080918400909171
S12340A08500880F991F880F991F9093850080938400CC0FDD1FCC0FDD1FD093CF03C09364
S12340C0CE038091260690912706880F991F880F991F9093270680932606809126069091F5
S12340E027060E94D81B9093B6078093B5078091F8059091F90583FF3AC0E091A704F09105
S1234100A804CF0183709070892B99F4209126063091270680912606909127066AE070E0FB
S12341200E94B32A261B370B3093B6072093B50718C020913A01809126069091270668E2F1
S123414070E00E94B32A30E0629FC001639F900D729F900D11248C599F4F9093B607809372
S1234160B5073196F093A804E093A70404C01092A8041092A70480914F04909150048A5851
S1234180924038F08091EA039091EB038E3691053CF48CE291E09093C0078093BF0704C024
S12341A01092C0071092BF078091B5079091B60720911601309117014091BF075091C0079F
S12341C0821B930B841B950B9093AC078093AB078091AB079091AC0797FF20C08091AB07F6
S12341E09091AC0720912606309127064091B5075091B607820F931F8417950778F420915A
S12342002606309127068091B5079091B607821B930B44969093AC078093AB07F894809188
S12342209507833011F48EE005C080919507843081F487E18093FC05809126069091270616
S12342400E94921E909389008093880081E0809396077894DF91CF911F910F9108951F9236
S12342600F920FB60F9211242F933F934F935F936F937F938F939F93AF93BF93EF93FF9386
S12342804B9926C0E0919507F0E08091B4039091B503EE0FFF1FE956F84F918380830E9478
S12342A0A51E0E94F7198091580490915904880F991F9093590480935804809158049091CE
S12342C0590481609093590480935804479822C220918400309185008091CA039091CB03A2
S12342E0969587952817390770F480914F0490915004815D974038F081E090E09093590489
S12343008093580407C28091F8059091F90583FFA2C080918400909185009093CB03809311
S1234320CA0310928500109284008091580490915904880F991F9093590480935804479A55
S123434020913A01809126069091270668E270E00E94B32A30E0629FC001639F900D729F47
S1234360900D11248C599F4F9093B6078093B50780914F04909150048051974208F057C053
S1234380809168079091690793FD51C08091B5079091B60790938B0080938A002091260694
S12343A03091270680912606909127069695879596958795281B390B3093220620932106A6
S12343C080919507813021F080919507843031F4449883E08093A50481E01BC08091950700
S12343E0853021F080919507823031F4459881E08093A50482E00DC080919507833021F0D5
S123440080919507863039F4469882E08093A50483E08093B7078EEB90E09093240680938F
S1234420230680916807909169079F770FC080912606909127068C509E4F90938B00809344
S12344408A008091680790916907906890936907809368075FC18091E80387FF5CC08091E1
S1234460A604882309F457C08091B4039091B5039093B7038093B6031092B5031092B403D2
S123448080918400909185009093CB038093CA0310928500109284008091580490915904D4
S12344A0880F991F9093590480935804479A1092A50480E09AEF90938B0080938A00809149
S12344C08A0090918B00909322068093210680919507813021F080919507843011F481E0E7
S12344E013C080919507853021F080919507823011F482E009C080919507833021F0809161
S12345009507863029F483E08093B7071092A50486E990E0F0C08091B4039091B503909356
S1234520B7038093B6031092B5031092B40380918400909185009093CB038093CA03109290
S12345408500109284008091580490915904880F991F9093590480935804479A80914F043E
S1234560909150048051974208F0CAC08091AB079091AC0785369105B4F11092A5048091AD
S1234580AB079091AC0790938B0080938A0080918A0090918B009093220680932106809169
S12345A09507813021F080919507843011F481E013C080919507853021F08091950782302D
S12345C011F482E009C080919507833021F080919507863029F483E08093B7071092A50437
S12345E084E090E088C08091AB079091AC078B5B9F4FF4F11092A50484E690E090938B0078
S123460080938A00909322068093210680919507813021F080919507843029F481E0809313
S1234620B707459819C080919507853021F080919507823029F482E08093B70746980CC036
S123464080919507833021F080919507863031F483E08093B70744981092A50488E290E028
S1234660909324068093230684E18093D00352C08091B5079091B60790938B0080938A005A
S123468020912606309127068091AB079091AC07820F931F9093220680932106809195073F
S12346A0813021F080919507843029F481E00E942E1A81E019C080919507853021F08091AD
S12346C09507823029F482E00E942E1A82E00CC080919507833021F080919507863031F4F8
S12346E083E00E942E1A83E08093A50484E18093D00384EB90E090932406809323060AC0CD
S123470080912606909127068C509E4F90938B0080938A002B9A7894FF91EF91BF91AF9185
S12347209F918F917F916F915F914F913F912F910F900FBE0F901F9018951092800081EFBC
S12347409FEF909389008093880085EF9FEF90938B0080938A0080E88093810080EC9AED44
S1234760909385008093840083E090E09093CD038093CC038091CC039091CD038068809382
S1234780810080916F00876080936F00539852983D9A3E9A459A469A449AA2E0B2E00E94D4
S12347A0172B802D8093B803A1E0B2E00E94172B802D8093B9038091B9038E3039F0809100
S12347C0B903873119F087E18093B903809169008460809369008091690081608093690070
S12347E0E99A089521EB30E0F90110821092B6001092B2001092B300A0E7B0E08C918360D5
S12348008C9338984098399841983A9842983B984398389839983A983B98EFE6F0E08081DD
S12348208D7F80838C918C7F8C9386E0F901808384E680931D060895813099F438983B989D
S123484080912D01843021F439983A981092D2031092C9071092C8071092D1031092B10086
S12348600895823049F439983A981092C7071092C6071092D20315BC08951F920F920FB62A
S12348800F9211242F933F934F935F936F937F938F939F93AF93BF93EF93FF93F894809129
S12348A0D103843019F481E00E941C247894FF91EF91BF91AF919F918F917F916F915F9120
S12348C04F913F912F910F900FBE0F901F9018950F931F938091EA039091EB030A9714F4F3
S12348E087E003C08091620486E08093B1001092B20080914F0490915004845F914018F4FC
S12349001092B40716C080914F04909150048D56974020F08EE08093B4070BC080914F0452
S12349209091500464E670E00E94B32A65506093B407E091B407F0E0E351FE4F80818093F1
S1234940130180916204882329F02091CC048091180109C0E0915304F0915404E854FB4F69
S1234960808120911801829FC00111249093AA048093A90480914F0490915004805991403D
S123498050F5809100019091010182FF1AC08091A9049091AA0420911901820F911D909384
S12349A0AA048093A90480916807909169078460909369078093680780911A018093AB048D
S12349C041C080916807909169078B7F909369078093680737C080916807909169078B7F90
S12349E090936907809368078091AB04823050F18091AB0481508093AB04E091A904F091F9
S1234A00AA04509119012091190180911A014091AB0460911A01E50FF11D90E0841B9109BB
S1234A2030E070E0AC01429FC001439F900D529F900D11240E94B32AE61BF70BF093AA04CE
S1234A40E093A90480916204882309F0EAC08091BB0787FD40C08091BB078331E4F5E09145
S1234A605304F0915404E754FB4F6081E0915304F0915404E854FB4F40810091A9041091D5
S1234A80AA0480918F072091BB07E091180170E0641B710990E04AE0240290011124821B54
S1234AA0930B9C01629FC001639F900D729F900D11246AE070E00E94C72AF0E06E9FC001A8
S1234AC06F9F900D7E9F900D1124800F911F9093AA048093A9048091910787FD40C080912A
S1234AE091078F30E4F5E0915304F0915404E453FB4F6081E0915304F0915404E854FB4F58
S1234B0040810091A9041091AA048091B80720919107E091180170E0641B710990E04AE0BD
S1234B20240290011124821B930BAC01649FC001659F900D749F900D11246AE070E00E9417
S1234B40C72AF0E06E9FC0016F9F900D7E9F900D1124800F911F9093AA048093A904809147
S1234B6000019091010184FF5CC020911604309117048091F6039091F70328173907FCF433
S1234B808091F6039091F7032091160430911704821B930B64E070E00E94C72A8091550479
S1234BA0861710F460935504809155048A3018F089E080935504809126018093AC04309147
S1234BC0AC043430C8F08091A9049091AA04E0915504F0E0ED51FE4F2081820F911D909350
S1234BE0AA048093A90431503093AC048091680790916907806109C0109255041092AC0447
S1234C0080916807909169078F7E90936907809368078091F6039091F703909317048093E7
S1234C201604809100019091010191FD09C08091E80386FF94C080916204882309F48FC087
S1234C4080911F068F5F80931F0690911F0680912006981708F486C010921F068091F203B9
S1234C609091F303E0919107FF27E7FDF095E350FA4F208130E02817390734F480911D0679
S1234C8090911E06890F19C08091F2039091F303E0919107FF27E7FDF095E350FA4F208188
S1234CA030E0821793075CF480911D0618163CF480911D0690911E06891B80931D06809167
S1234CC06807909169079D7F909369078093680720911D06E0919107FF27E7FDF095E35000
S1234CE0FA4F8089332727FD309590E08C599F4F8217930754F4E0919107FF27E7FDF095C5
S1234D00E350FA4F80898C591EC020911D06E0919107FF27E7FDF095E350FA4F408933273C
S1234D2027FD309584E690E0841B910928173907CCF4E0919107FF27E7FDF095E350FA4F20
S1234D40908984E6891B80931D0680916807909169079260909369078093680703C084E6AD
S1234D6080931D068091A9049091AA0420918E0730E062E070E00E94C72A269FC001279FA5
S1234D80900D369F900D112464E670E00E94B32A660F771F7093AA046093A90420910004A1
S1234DA03091010480911C0190E0C296281739070CF04DC0809100019091010181FF47C0EF
S1234DC08091000490910104C397D4F040911B0180911B01209100043091010460911C01D3
S1234DE090E070E06E5C7F4FFC01E29FC001E39F900DF29F900D11240E94B32A461B03C0F3
S1234E0080911B01482F50E08091A9049091AA04480F591F5093AA044093A904189905C0D7
S1234E20809121019091220104C080911D0190911E019093200180931F01809168079091AC
S1234E4069078260909369078093680711C080916807909169078D7F9093690780936807E4
S1234E6080911D0190911E019093200180931F018091F8059091F90583FF1CC0E091A9049F
S1234E80F091AA0420913B018091A9049091AA0464E170E00E94C72A30E0629FC001639F69
S1234EA0900D729F900D11248E0F9F1F9093AA048093A904809100019091010190FF4CC0B2
S1234EC08091EA039091EB03823891050CF044C08091A9049091AA0420912801820F911DCB
S1234EE09093AA048093A904E091EA03F091EB03609118012091280182E890E08E1B9F0B3F
S1234F0070E0AB01849FB001859F700D949F700D11248FEF90E0FB01E89FB001E99F700D10
S1234F20F89F700D1124882777FD8095982F30E040E050E00E94882A20E43FE140E050E0FD
S1234F400E94DA2A8091A9049091AA04820F931F9093AA048093A9042091A9043091AA0479
S1234F608091180145EF849FC00111248217930754F480911801849FC00111249093AA0427
S1234F808093A9040BC08091A9049091AA041816190624F01092AA041092A9048091A90437
S1234FA09091AA04909357048093560478941F910F9108951F920F920FB60F9211242F938B
S1234FC03F934F935F936F937F938F939F93AF93BF93EF93FF93F8942091D103223039F08B
S1234FE0243009F44FC0213009F051C01CC08091C8079091C9078F3F9105D1F1C8F1809155
S1235000C8079091C9078F5F8093B3008091C8079091C9078F5F90409093C9078093C807B4
S12350202093D10334C00E94682480915604909157049093C9078093C8078091C807909106
S1235040C9078F3F9105A1F098F08091C8079091C9078F5F8093B3008091C8079091C907A9
S12350608F5F90409093C9078093C80782E007C08091C8079091C9078093B30084E0809362
S1235080D10305C081E00E941C241092D1037894FF91EF91BF91AF919F918F917F916F91AE
S12350A05F914F913F912F910F900FBE0F901F9018951F920F920FB60F9211242F933F93A4
S12350C04F935F936F937F938F939F93AF93BF93EF93FF93F8942091D203223039F0243007
S12350E009F453C0213009F053C020C08091C6079091C7078F3F910591F088F08091C60757
S12351009091C7078F5F87BD8091C6079091C7078F5F90409093C7078093C60733C080910A
S1235120C6079091C70787BD84E024C080915604909157049093C7078093C60724E025BD85
S123514016BC8091C6079091C7078F3F9105A9F0A0F08091C6079091C7078F5F87BD80910F
S1235160C6079091C7078F5F90409093C7078093C60782E08093D2030BC08091C6079091CC
S1235180C70787BD2093D20303C082E00E941C247894FF91EF91BF91AF919F918F917F915E
S12351A06F915F914F913F912F910F900FBE0F901F9018951F920F920FB60F9211242F9375
S12351C03F934F935F936F937F938F939F93AF93BF93EF93FF93F8948091D203843019F4E2
S12351E082E00E941C247894FF91EF91BF91AF919F918F917F916F915F914F913F912F91FB
S12352000F900FBE0F901F90189554985C9855985D985498559815BCEEE6F0E0808183602F
S1235220808384E085BD16BC82E187BD089511B88FEF84B915B887B98AB908950895089500
S12352400895089588E98093C10083E18093C40081E198E09093CF078093CE079093CB07E0
S12352608093CA0781ED97E09093CD078093CC0790935208809351081092D0071092250655
S123528008951F920F920FB60F9211248F939F93EF93FF938091D007882311F1E091CE073D
S12352A0F091CF0781918093C600F093CF07E093CE07E155F84030F081E198E09093CF07A6
S12352C08093CE078091D00781508093D0078091D007882329F48091C1008F7D8093C100DD
S12352E0FF91EF919F918F910F900FBE0F901F9018951F920F920FB60F9211242F938F9312
S12353009F93EF93FF938091C600E0915108F09152088083809125068F5F8093250680914B
S1235320510890915208019690935208809351088151984030F081ED97E0909352088093D6
S12353405108FF91EF919F918F912F910F900FBE0F901F90189580912506882319F48FEFF7
S12353609FEF0895F89480912506815080932506E091CC07F091CD072191F093CD07E09312
S1235380CC07E151F84030F081ED97E09093CD078093CC077894822F90E00895982F809148
S12353A0D0078F33E0F78091D007803418F080E090E00895F8948091D0078F5F8093D0071C
S12353C0E091CA07F091CB0790838091CA079091CB0701969093CB078093CA07815598402E
S12353E030F081E198E09093CB078093CA078091C10080628093C100789481E090E00895D4
S1235400CF93DF93EC0104C00E94CE298111219688818823C9F781E090E0DF91CF9108956F
S123542083ED93E00E94002A08958BED93E00E94002A08958091250690E00895CF92DF92AD
S1235440EF92FF920F931F93CF93DF93CDB7DEB729970FB6F894DEBF0FBECDBF8C01F62E3D
S1235460E42EDE011196EEEDF3E089E001900D928150E1F749E06E010894C11CD11CFF2083
S123548081F089E090E0841B91092F2D30E08217930738F04150F601E40FF11D8CE28083C4
S12354A0FF244150F601E40FF11DC8016AE070E00E94B32A805D8083C8016AE070E00E9475
S12354C0B32A8B01672B11F4FF2019F085E08F15B0F619E01E197E010894E11CF11C07C0D5
S12354E0F701E10FF11D80810E94CE291F5F1930B8F329960FB6F894DEBF0FBECDBFDF9130
S1235500CF911F910F91FF90EF90DF90CF900895629FD001739FF001829FE00DF11D649F6A
S1235520E00DF11D929FF00D839FF00D749FF00D659FF00D9927729FB00DE11DF91F639F68
S1235540B00DE11DF91FBD01CF0111240895991B79E004C0991F961708F0961B881F7A957F
S1235560C9F780950895AA1BBB1B51E107C0AA1FBB1FA617B70710F0A61BB70B881F991F21
S12355805A95A9F780959095BC01CD01089597FB092E07260AD077FD04D0E5DF06D0002044
S12355A01AF4709561957F4F0895F6F7909581959F4F0895A1E21A2EAA1BBB1BFD010DC08F
S12355C0AA1FBB1FEE1FFF1FA217B307E407F50720F0A21BB30BE40BF50B661F771F881F63
S12355E0991F1A9469F760957095809590959B01AC01BD01CF01089597FB092E05260ED067
S123560057FD04D0D7DF0AD0001C38F450954095309521953F4F4F4F5F4F0895F6F79095C8
S12356208095709561957F4F8F4F9F4F0895F999FECFB2BDA1BDF89A119600B40895F7DF93
S1235640E02DF5DFF02D0895F999FECFB2BDA1BD00BC11960FB6F894FA9AF99A0FBE08953A
S1235660F3DF012CF1DF11240895FFCF2F000100020003000400050006000700080032280A
S1235680E803900106141E1E3C581B581B88136419121E01010203040A0411C4098813C474
S12356A0096400DCE64003020A14324696280000000000000000000000000000000000001E
S12356C00000000000000000000000000000000000000000000000000000000000000000C6
S12356E00000000000000000000000000000000102030405060708090A0B0C0D0E0F10011D
S123570002030405060708090A0B0C0D0E0F100102030405060708090A0B0C0D0E0F101462
S1235720161718191A1B1C1D1E1F2021222324191A1B1C1D1E1F2021222324252627271E8D
S12357401F2022232425262728292A2B2C2D2E000204060708090A0C0E28262422201E1EC6
S12357601E1E1E1E1E1E1E1E1EF0FF80BBE0880465484BA438022BF0207019CC13860F442F
S12357800CC209D0074C061B052A046A03D1025602F201A1015F012801FB00D600B7009DDC
S12357A00087007500660059004D0044003C0034002E0029002500F0FF80BBE0880465486A
S12357C04BA438022BF0207019CC13860F440CC209D0074C061B052A046A03D1025602F248
S12357E001A1015F012801FB00D600B7009D0087007500660059004D0044003C0034002E6A
S12358000029002500F0FF80BBE0880465484BA438022BF0207019CC13860F440CC209D0A7
S1235820074C061B052A046A03D1025602F201A1015F012801FB00D600B7009D00870075E6
S123584000660059004D0044003C0034002E0029002500F0FF80BBE0880465484BA438029C
S12358602BF0207019CC13860F440CC209D0074C061B052A046A03D1025602F201A1015FCE
S1235880012801FB00D600B7009D0087007500660059004D0044003C0034002E002900257D
S12358A0000000F5047E05AE066C08C00AB30D630F8B10D7118813000000000A000F001EEF
S12358C0003C007800FA007201E00180028002000008000A000C000E00C80A4A067E04846A
S12358E003AC0D641A002000270032003E0066008E00B202EB02240337034B0356036103B2
S12359007003E800D600C200B0009D008A00780078006500520040002D0019000700000085
S12359200100010001175A5A5A505050505050505050505050506400030000FA3204041B75
S11759405B481B5B324A000D0A002020202020202020200083
S50302CB2F
